:020000040000FA
:020000000428D2
:08000800FF30A200FF30A3004D
:100010008B0107309F00FF30132100301121003089
:100020000C210130A5000130A600A0102011051CF4
:100030001C28A01C1E284528A01C4528A010051C13
:100040002228A01405184528851C3628051E2F28AF
:100050002608AC202708A6002608FA2035282608FE
:10006000F0202708A6002608FA204528051E3F286C
:10007000260875202708A6002608FA204528260805
:10008000E3202708A6002608FA20051D4A28201D7F
:100090004C287328201D73282011051D5028201579
:1000A00005197328851D6428051E5D282508AC20C8
:1000B0002708A5002508032163282508F020270824
:1000C000A500250803217328051E6D282508752025
:1000D0002708A5002508032173282508E320270801
:1000E000A5002508032117287428A7000F30A705AD
:1000F0002708083C031D7F280C30A700AB282708E1
:100100000C3C031D86280430A700AB282708043CBC
:10011000031D8D280630A700AB282708063C031DC9
:1001200094280230A700AB282708023C031D9B2817
:100130000330A700AB282708033C031DA228013089
:10014000A700AB282708013C031DA9280930A700F8
:10015000AB280830A7000800A7000F30A705270824
:10016000013C031DB6280330A700E2282708033C02
:10017000031DBD280230A700E2282708023C031D0A
:10018000C4280630A700E2282708063C031DCB2818
:100190000430A700E2282708043C031DD2280C30B5
:1001A000A700E22827080C3C031DD9280830A70027
:1001B000E2282708083C031DE0280930A700E228B0
:1001C0000130A7000800A700271CEB280310270C0C
:1001D0000838A700ED280310A70C0F30A70508006A
:1001E000A7000310A70D271EF7280130A7040F3022
:1001F000A7050800A700270EF039A80024080F392A
:100200002804A4000E29A70027080F39A8002408F5
:10021000F0392804A4000E29A4000E292408860021
:100220000800A3001529A200192923081D21860012
:10023000202922081D218500202983160313080088
:0602400083120313080005
:02400E00623F0F
:00000001FF
